:100000000C94BB020C9402030C9402030C940203A4
:100010000C9402030C9402030C9402030C9402034C
:100020000C9402030C9402030C94D20C0C94A40DB7
:100030000C9402030C9402030C9402030C9402032C
:100040000C9402030C94EC220C9402030C94020313
:100050000C9402030C947C1C0C9402030C94020379
:100060000C9402030C9402030C9402030C940203FC
:100070000C9402030C9402030C9402030C940203EC
:100080000C9402030C9402030C9402030C940203DC
:100090000C9402030C9402030C9402030C940203CC
:1000A0000C9402030C9402030C940203110E330E01
:1000B000210F330E210F780E9B0E210FF00E030F30
:1000C000EF11EF112C122C126F12AD12C614C614C0
:1000D000C612C614C713C7139A14C614C614B11493
:1000E0000000F0A1F0A2F0A335822B77297FE10078
:1000F000508100001E00140004001D004F834D833A
:100100001F001A0016001B00E0004C002000080031
:1001100007000600E2002A0021001500090019006E
:10012000E3004A81220017000A0005000000E000F9
:100130002C082F0000002B000000E3002D003000F1
:1001400000002B020000E30423001C000B00110040
:100150000000E302240018000D001000E7004B82AD
:1001600025000C000E00360052002C002600120064
:100170000F00370051002800270013003382388217
:10018000C3004E812E003177347FE500C1000000AE
:100190000100010001000100010000003A001E0200
:1001A00020022202010001003B001F022102230263
:1001B000010001003C002F0226022F000100010077
:1001C0003D00300227023000010001003E003102F4
:1001D0003500350200000100010036020000690010
:1001E000000001002B00370200006A00000001003F
:1001F0003F003302330024020000010040002400CD
:1002000021001E00270001004100250022001F00E0
:100210003700010042002600230020002E000100CC
:100220004300310025022D002E020100440045004C
:100230000100280001000000010001000100010090
:10024000010000000100140801001D080100010068
:1002500001001A0801001B08010001000100010053
:100260000100060801000100010001000100190859
:100270000100010001000100010006010000010071
:1002800001002B0200000100000001000100AE008F
:100290000000A800000001000100AC00AA0001005D
:1002A000000001000100AB00A900010001000100F5
:1002B0000100010001000100010001000100010036
:1002C00001000100010001000100460001000100E1
:1002D0000100010001000100010001000100000017
:1002E000A500010001000100010000000100010063
:1002F000010001000100010001000100F200010005
:10030000010001000100F000F10001000100010006
:1003100001000100F30001000100E2000100010002
:10032000F400F5000000E100010001000000010000
:1003300000000100010001000000010000004A006F
:10034000010001005000010000004D00010001000B
:1003500051000100010001000100010052000100F4
:1003600001000100010001004F0001000100010037
:100370000100010001000100010001000100010075
:100380000100010001000000160345007200670033
:100390006F0044006F007800200045005A00000004
:1003A00016034500720067006F0044006F0078007C
:1003B000200045005A0000000403090409026D00F2
:1003C000040100A0FA090400000103010100092151
:1003D00011010001223F000705810308000A0904FA
:1003E00001000103010200092111010001224D0059
:1003F0000705820308000A09040200010300000047
:100400000921110100012236000705830308000AB3
:100410000904030001030000000921110100012269
:1004200039000705840310000112011001000000CB
:1004300008EDFE071301000102000105010906A1F4
:1004400001050719E029E7150025019508750181C7
:100450000205081901290595057501910295017597
:100460000391010507190029771500250195787575
:10047000018102C005010980A10185021601002643
:10048000B7001A01002AB700751095018100C00558
:100490000C0901A1018503160100269C021A010026
:1004A0002A9C02751095018100C005010902A10175
:1004B0000901A10005091901290515002501950566
:1004C000750181029501750381010501093009312A
:1004D0001581257F95027508810609381581257FCC
:1004E000950175088106050C0A38021581257F954E
:1004F0000175088106C0C005010906A1010507199B
:10050000E029E7150025019508750181029501751F
:1005100008810105081901290595057501910295C4
:1005200001750391010507190029FF150025FF95A5
:100530000675088100C000000000000000000000F7
:1005400000010204060A0F17202C3A4A5D71879DAC
:10055000B3C7DAE9F5FCFFFCF5E9DAC7B39D8771AB
:100560005D4A3A2C20170F0A060402010000000021
:1005700000000000000011241FBECFEFDAE0DEBF54
:10058000CDBF04B603FE27C08091260290912702BA
:10059000A0912802B09129028730904BA740B04B20
:1005A000D1F4109226021092270210922802109283
:1005B000290214BE84B7877F84BF0FB6F894A8952C
:1005C00080916000886180936000109260000FBE8F
:1005D000E0E0FFE3099511E0A0E0B1E0E4E8F9E430
:1005E00002C005900D92A433B107D9F722E0A4E32D
:1005F000B1E001C01D92A632B207E1F70E94130AD2
:100600000C94C0240C94000061110BC0FC01828189
:10061000882321F085EE0E94831003C085EE0E949E
:100620004B1180E090E0089508956091E901709188
:10063000EA018091EB019091EC010E94A51B569874
:100640005E9825982D9826982E9827982F98823076
:1006500039F0833041F0813041F4259A2D9A089584
:10066000269A2E9A0895279A2F9A08950C94150386
:1006700056985E9825982D9826982E9827982F980A
:100680008FEF90E0909389008093880090938B0087
:1006900080938A0090938D0080938C00259A2D9AE8
:1006A0002FEF80E792E0215080409040E1F700C0BA
:1006B0000000269A2E9A2FEF80E792E0215080408A
:1006C0009040E1F700C00000279A2F9A2FEF80E7B3
:1006D00092E0215080409040E1F700C00000259852
:1006E0002D982FEF80E792E0215080409040E1F775
:1006F00000C0000026982E982FEF80E792E021504E
:1007000080409040E1F700C0000027982F9856984D
:100710005E9825982D9826982E9827982F980895BA
:1007200089EA8093800089E08093810024982C9846
:100730003F988AB18F748AB96E98479A8BB1806B53
:100740008BB9769A0E9438030C94140380E280934C
:1007500000018091340181110EC00E94F50381E0F7
:10076000809334012FEF83ED90E32150804090403F
:10077000E1F700C0000080E40E94FB0380930001C9
:1007800081112EC00E94250480930001811128C090
:100790000E94250480930001811122C08FE30E94F2
:1007A00025048093000181111BC00E941D0480E478
:1007B0000E94FB0380930001811112C08CE00E9413
:1007C00025048093000181110BC00E9425048093B1
:1007D0000001811105C08FE30E9425048093000170
:1007E0000E941D048091000108951092B9008AE0D2
:1007F0008093B800089594EA9093BC009091BC0057
:1008000097FFFCCF9091B900987F983021F09031FC
:1008100011F081E008958093BB0084E88093BC00D0
:100820008091BC0087FFFCCF8091B900887F883120
:1008300011F0803471F780E0089584E98093BC0062
:100840008091BC0084FDFCCF08958093BB0084E8B8
:100850008093BC008091BC0087FFFCCF9091B900D1
:10086000987F81E0983209F480E0089584E88093CD
:10087000BC008091BC0087FFFCCF8091BB00089535
:1008800080910001811115C080E40E94FB038093D8
:10089000000181110CC082E10E94250480930001B7
:1008A000811105C08FEF0E942504809300010E94F2
:1008B0001D0484B1807F84B985B1807F85B98AB1F8
:1008C000837F8AB98BB1837F8BB93E984698089510
:1008D0000E94A603809300010E94400480B38C70A4
:1008E00080BB81B3836F81BBA6E3B1E0E4E4F1E0B8
:1008F0008EE08E0F11921D928E13FCCF0C949003FC
:10090000BF92CF92DF92EF92FF920F931F93CF93FC
:10091000DF9380910001882379F0809135018F5F0A
:1009200080933501811108C00E94A60380930001C5
:10093000811102C00E94380306E311E0C0E0D0E05C
:10094000DD24D39482E0C82EEE24E394F12CC7304A
:10095000D10500F580910001811164C080E40E94FE
:10096000FB0380930001811112C082E10E942504E3
:100970008093000181110BC0C7010C2E01C0880FAC
:100980000A94EAF780950E942504809300010E9452
:100990001D0448C0CA30A1F028F4C83059F0C9304D
:1009A00061F005C0CC3089F070F0CD3089F0209A2C
:1009B000289810C0219A29980DC0229A2A980AC016
:1009C000239A2B9807C0529A01C0539A5B9802C091
:1009D0003E9A469890EA9A95F1F79FB1799902C0AC
:1009E00082E001C080E091709D25982B7C9902C027
:1009F00084E001C080E0892B7D9902C038E001C00D
:100A000030E0832B7E9902C020E101C020E0822BE0
:100A10009FB19095991F9927991F9295990F907E54
:100A2000892B0FC080910001811149C080E40E9490
:100A3000FB0380930001882379F1B12C0E941D04EF
:100A40008B2DF8019081981719F08083C0920101D5
:100A50000E94400421960F5F1F4FCE30D10509F050
:100A600076CF80910101882361F18150809301014B
:100A7000882339F08FE99FE00197F1F700C000006B
:100A800020C0A4E4B1E0E6E3F1E0CF01825F919100
:100A90009D938E13FCCF15C083E10E9425048093A3
:100AA00000018111CACF81E40E94FB038093000101
:100AB0008111C3CF0E943604B82EB094BFCF80E01E
:100AC000C0CF0E94360381E0DF91CF911F910F913B
:100AD000FF90EF90DF90CF90BF900895E82FF0E067
:100AE000EC5BFE4F808108950895089596E0799F0C
:100AF000F001112494E5899FE00DF11D1124E60F0A
:100B0000F11DEE0FFF1FE851FF4F8591949108955D
:100B1000880F991FFC01E05AF04085919491089547
:100B2000880F991FFC01E052FF4F85919491089521
:100B30000F931F93CF93DF93EC018115904350F5F2
:100B4000C11580E2D80708F0B3C0CB3BD10590F4C3
:100B5000C83AD10508F05AC0C53AD10508F04BC0D3
:100B6000C430D10508F0BBC1219709F0B5C101E03F
:100B700010E0F5C1CF3FD10511F008F0B0C1C03F82
:100B8000D10508F092C0CE01805E9109089708F463
:100B9000A6C1A2C1C11591E5D907A8F4C23020E5CC
:100BA000D20708F09EC0C11580E5D80709F485C0BA
:100BB00008F091C0C11520E4D20708F08DC1DD27EF
:100BC0008E01106CCCC1C11580E8D80758F4C1154E
:100BD00090E7D90708F07CC1C11520E6D20708F4D8
:100BE00022C17AC1C11580E9D80708F075C1DF704C
:100BF0008E01106AB4C1C53AD10509F472C1C63A72
:100C0000D10509F071C102E810E4A9C1C83AD105C3
:100C100009F46DC1C93AD10509F46CC1CA3AD105CC
:100C200009F46BC1CB3AD10509F46AC1CC3AD105BC
:100C300009F469C1CD3AD10509F468C1C03BD105B9
:100C400009F467C1CE3AD10509F466C1CF3AD1059E
:100C500009F465C1C13BD10509F464C1C23BD105AA
:100C600009F463C1C33BD10509F462C1C43BD1059A
:100C700009F461C1C53BD10509F460C1C63BD1058A
:100C800009F45FC1C73BD10509F45EC1C83BD1057A
:100C900009F45DC1C93BD10509F45CC1CA3BD1056A
:100CA00009F45BC100E014E45AC18E01106557C11C
:100CB000CE019F700E94900553C10E94EA149FEFDD
:100CC00024E38CE0915020408040E1F700C0000018
:100CD0000E94A11C44C1809105028160809305029D
:100CE0003EC10E944A1E811102C00E94301E0E9415
:100CF000671E90E09093260280932502C23090E513
:100D0000D90721F480912502816086C0C43020E596
:100D1000D20721F48091250282607EC0C63080E532
:100D2000D80721F480912502846076C0C83090E510
:100D3000D90719F48091250227C0CA3020E5D207CF
:100D400021F480912502806167C0CC3080E5D8070E
:100D500021F48091250280625FC0CE3090E5D907F2
:100D600021F480912502806457C0C03120E5D2076C
:100D700021F48091250280684FC0C23180E5D807F8
:100D800029F4809125028460886046C0C33090E5D4
:100D9000D90721F4809125028E7F3EC0C53020E521
:100DA000D20721F4809125028D7F36C0C73080E5BF
:100DB000D80721F4809125028B7F2EC0C93090E5A1
:100DC000D90719F48091250226C0CB3020E5D2073F
:100DD00021F4809125028F7E1FC0CD3080E5D80799
:100DE00021F4809125028F7D17C0CF3090E5D9077F
:100DF00021F4809125028F7B0FC0C13120E5D207FD
:100E000021F4809125028F7707C0C331D04531F49A
:100E1000809125028B7F877F809325028091250218
:100E20000E946B1E9CC08D2F99278F70992781304F
:100E30009105D9F49E012370332702C0880F991FB2
:100E40002A95E2F79C688E0144E0000F111F4A9535
:100E5000E1F700271370802B912B53E0CC0FDD1F9F
:100E60005A95E1F7C076DD272FC08230910531F425
:100E7000DC2FCC278E01016F106A71C08330910581
:100E800069F4CE018370992701E010E002C0000FE1
:100E9000111F8A95E2F7C8019C680FC0049709F0FA
:100EA0005EC0CE018370992701E010E002C0000F00
:100EB000111F8A95E2F7C8019A6823E0CC0FDD1F65
:100EC0002A95E1F7C07ED7708C010C2B1D2B47C0F3
:100ED000DF708E01106243C000E010E040C08E0160
:100EE0003EC001E810E43BC003E810E438C002EE65
:100EF00014E435C009EE14E432C00AEE14E42FC045
:100F000005EB14E42CC006EB14E429C007EB14E451
:100F100026C00CEC14E423C00DEC14E420C003E85C
:100F200015E41DC00AE815E41AC002E915E417C06B
:100F300004E915E414C001E216E411C003E216E46A
:100F40000EC004E216E40BC005E216E408C006E297
:100F500016E405C007E216E402C00AE216E4C8017E
:100F6000DF91CF911F910F91089596E0799FF00145
:100F7000112494E5899FE00DF11D1124E60FF11D68
:100F8000EE0FFF1FE851FF4F85919491803E910530
:100F9000E0F4803C910558F58133910509F46FC068
:100FA00048F48932910509F463C08A32910509F445
:100FB0006DC072C089339105E9F082389105D1F096
:100FC0008533910509F44DC067C0833E910581F1D9
:100FD00038F4803E9105B9F0823E9105D9F05CC0AD
:100FE000863E910561F1873E9105A1F155C00E94B1
:100FF000880508952091250220FD02C021FF4CC0E4
:1010000080EE90E049C08091250280FFF9CF89E30E
:1010100090E042C08091250282FF0EC0809125029F
:1010200084FF03C080E090E037C083EE90E034C0DE
:101030008091250282FFF2CF82EE90E02DC0809158
:10104000250283FF0BC08091250284FDEBCF87EE44
:1010500090E022C08091250283FFF5CF86EE90E0DC
:101060001BC08091250285FF07C089E290E014C073
:101070008091250285FFF9CF85E390E00DC0809136
:10108000250286FF07C08AE290E006C08091250213
:1010900086FFF9CF81E390E00E94980508950895B6
:1010A0000C944F08809162010895CF93DF9300D094
:1010B0001F92CDB7DEB79C0180911C02843019F5D8
:1010C00093E099833B832A839093E9008FEF90917B
:1010D000E800815095FD06C095ED9A95F1F7000066
:1010E0008111F5CF8091E80085FF0DC040E050E010
:1010F00063E070E0CE0101960E94C20A8091E80090
:101100008E778093E8000F900F900F90DF91CF9132
:101110000895CF93DF9300D01F92CDB7DEB7209113
:101120001C02243021F522E029839B838A8383E0FB
:101130008093E9008FEF9091E800815095FD06C003
:1011400095ED9A95F1F700008111F5CF8091E800B7
:1011500085FF0DC040E050E063E070E0CE010196F5
:101160000E94C20A8091E8008E778093E8000F9079
:101170000F900F90DF91CF91089520911C022430A1
:10118000F1F422E02093E9002FEF3091E8002150A4
:1011900035FD06C035ED3A95F1F700002111F5CF88
:1011A0002091E80025FF0BC040E050E065E070E0D2
:1011B0000E94C20A8091E8008E778093E80008952B
:1011C000CF93DF93EC0190911C02943009F046C05C
:1011D00080910C018823D9F080910D018823B9F00A
:1011E0009093E9008FEF9091E800815095FD06C043
:1011F00095E19A95F1F700008111F5CF8091E80013
:1012000085FF2CC040E050E060E170E017C081E055
:101210008093E9008FEF9091E800815095FD06C022
:1012200095ED9A95F1F700008111F5CF8091E800D6
:1012300085FF14C040E050E068E070E0CE010E94FD
:10124000C20A8091E8008E778093E80080E1FE0179
:10125000A2E5B1E001900D928A95E1F7DF91CF917F
:10126000089580911B02811109C00E94570C0E94B1
:10127000B40C8091E20084608093E20008951092A3
:101280001B02089508950C94D9220E94371C0E94D5
:10129000DF220E945A0F0C94500842E061EC81E07A
:1012A0000E94D10B42E061EC82E00E94D10B42E04F
:1012B00061EC83E00E94D10B42E161EC84E00C948C
:1012C000D10B80911E02833009F455C030F4813077
:1012D00071F0823009F48EC008958A3009F47AC022
:1012E0008B3009F460C0893009F09CC020C0809127
:1012F0001D02813A09F096C08091E800877F8093B3
:10130000E8008091210290912202892B21F460E172
:1013100082E591E003C060E080E090E070E00E9430
:101320000D0B8091E8008B778093E8000895809101
:101330001D02813209F076C0809121029091220233
:10134000009719F0039709F06DC08091E800877F3E
:101350008093E8008091E80082FD05C080911C0226
:101360008111F8CF5FC08091F1008093620180917C
:10137000E8008B7753C080911D02813A09F052C07A
:101380008091210290912202892B09F04BC080911B
:10139000E800877F8093E8008091E80080FFFCCF21
:1013A00080910C0136C080911D028132D9F5809167
:1013B000210290912202892BA9F58091E800877F74
:1013C0008093E8000E94060C80911F0280930C011C
:1013D0000C94EA1480911D02813221F58091E8007D
:1013E000877F8093E8000E94060C80912002809302
:1013F0006301089580911D02813AA1F48091E80073
:10140000877F8093E8008091E80080FFFCCF809187
:1014100063018093F1008091E8008E778093E8006B
:101420000C94060C089584B7877F84BF0FB6F89498
:10143000A8958091600088618093600010926000A0
:101440000FBE90E080E80FB6F8948093610090930F
:1014500061000FBE0E94A90F0E94570C0E94B40C9D
:101460008091E20084608093E20078940E943A0FB9
:101470000E94AB0F82E091E00E94550F0E94C722AC
:1014800080911C02853069F40E94F51B80911A023C
:101490008823B1F30E94231C882391F30E94AC0A95
:1014A000EFCF0E94B10FECCF292F33272330310526
:1014B000C9F064F42130310581F02230310509F0A2
:1014C00043C08DE690E02CEB33E042C02132310581
:1014D000F1F02232310541F137C082E190E029E29A
:1014E00034E036C099278130910541F08230910572
:1014F00041F0892B49F5E8EBF3E005C0E0EAF3E0C1
:1015000002C0E8E8F3E0849190E09F0121C06430DC
:10151000D8F4E62FF0E0EE0FFF1FEE5DFE4F2081C6
:10152000318189E090E014C0643070F470E0FB0118
:10153000EE0FFF1FE65EFE4F20813181FB01EA5E68
:10154000FE4F808190E004C080E090E020E030E039
:10155000FA0131832083089580E189BD82E189BD4C
:1015600009B400FEFDCF8091D8008F7D8093D80014
:101570008091E00082608093E0008091E00081FD36
:10158000FCCF0895CF92DF92EF92FF920F931F93BB
:10159000CF93DF93EC018B016A010E94250C81112E
:1015A00033C0C114D10439F0F60180819181081B48
:1015B000190BC80FD91FE12CF12C0115110519F1D8
:1015C0008091E80085FD16C08091E8008E778093B9
:1015D000E800C114D10449F0F60180819181E80E40
:1015E000F91EF182E08285E00FC00E94250C88235D
:1015F00021F30AC089918093F10001501109FFEF96
:10160000EF1AFF0ADACF80E0DF91CF911F910F919F
:10161000FF90EF90DF90CF900895209123023091BA
:1016200024022617370748F06115710539F4209117
:10163000E8002E772093E80001C0B90140E0611571
:101640007105A9F120911C02222309F443C0253021
:1016500009F442C02091E80023FD40C02091E80039
:1016600022FD32C02091E80020FFE9CF4091F30035
:101670002091F20030E0342BFC01CF01611571059F
:1016800059F02830310540F481918093F100615088
:1016900071092F5F3F4FF1CF41E02830310509F04C
:1016A00040E02091E8002E772093E800C8CF411158
:1016B000C9CF0AC080911C02882361F0853061F097
:1016C0008091E80083FD0AC08091E80082FFF2CF9C
:1016D00080E0089582E0089583E0089581E0089510
:1016E00020912302309124022617370748F0611514
:1016F000710539F42091E8002E772093E80001C0AD
:10170000B901FC0120E06115710591F180911C0285
:10171000882309F440C0853009F43FC08091E80077
:1017200083FD3DC08091E80082FD2FC08091E800DC
:1017300080FFE9CF2091F3008091F20090E0922B9E
:101740006115710559F08830910540F4249120937A
:10175000F1003196615071090196F2CF21E00897AE
:1017600009F020E08091E8008E778093E800CBCFED
:101770002111CCCF0AC080911C02882361F08530F2
:1017800061F08091E80083FD0AC08091E80082FF4B
:10179000F2CF80E0089582E0089583E0089581E02B
:1017A0000895982F973058F59093E900981739F0DD
:1017B0007091EC002091ED005091F00003C0242FB7
:1017C000762F50E021FF19C03091EB003E7F30931F
:1017D000EB003091ED003D7F3093ED003091EB0058
:1017E00031603093EB007093EC002093ED00509348
:1017F000F0002091EE0027FF07C09F5FD3CF8F70CE
:101800008093E90081E0089580E0089580911D02B1
:1018100087FF11C08091E80082FD05C080911C0205
:101820008111F8CF11C08091E8008B770BC08091B7
:101830001C02882349F08091E80080FFF8CF809156
:10184000E8008E778093E80008952091E4003091BD
:10185000E50095E64091EC00842F817040FF22C0A6
:101860008091E80080FD1CC080911C02882391F0CB
:10187000853091F08091EB0085FD10C04091E4002F
:101880005091E5004217530729F39A01915011F73F
:1018900084E0089582E0089583E0089581E008954A
:1018A00080E008954091E80042FFDECF08950E9455
:1018B000C50C0E94CD0CE0EEF0E080818160808359
:1018C000E8EDF0E080818F77808319BCA7EDB0E070
:1018D0008C918E7F8C9380818F7E808310921B02EF
:1018E00008950F931F93CF93DF930E94C50C0E941E
:1018F000CD0CC8EDD0E088818F778883888180689F
:10190000888388818F7D888319BC10921C02109275
:10191000180210921A021092190200EE10E0F8015B
:1019200080818B7F808388818160888342E060E052
:1019300080E00E94D10BE1EEF0E080818E7F808319
:10194000E2EEF0E080818160808380818860808326
:10195000F80180818E7F8083888180618883DF9118
:10196000CF911F910F910895E8EDF0E080818F7E77
:101970008083E7EDF0E080818160808384E082BF36
:1019800081E080931B020C94710CE8EDF0E0808103
:101990008E7F80831092E20008951092DA001092F8
:1019A000E10008951F920F920FB60F9211242F930A
:1019B0003F934F935F936F937F938F939F93AF93D7
:1019C000BF93EF93FF938091E10082FF0BC0809162
:1019D000E20082FF07C08091E1008B7F8093E100ED
:1019E0000E94390F8091DA0080FF1FC08091D800DB
:1019F00080FF1BC08091DA008E7F8093DA00809197
:101A0000D90080FF0DC080E189BD82E189BD09B4A4
:101A100000FEFDCF81E080931C020E94310905C0C9
:101A200019BC10921C020E943F098091E10080FFC6
:101A300019C08091E20080FF15C08091E2008E7F86
:101A40008093E2008091E20080618093E2008091C7
:101A5000D80080628093D80019BC85E080931C0276
:101A60000E9443098091E10084FF30C08091E20030
:101A700084FF2CC080E189BD82E189BD09B400FEEC
:101A8000FDCF8091D8008F7D8093D8008091E100B8
:101A90008F7E8093E1008091E2008F7E8093E20050
:101AA0008091E20081608093E20080911802882397
:101AB00011F084E007C08091E30087FD02C081E05F
:101AC00001C083E080931C020E9445098091E100DF
:101AD00083FF29C08091E20083FF25C08091E1004F
:101AE000877F8093E10082E080931C0210921802AD
:101AF0008091E1008E7F8093E1008091E2008E7FF3
:101B00008093E2008091E20080618093E20042E0F5
:101B100060E080E00E94D10B8091F00088608093AB
:101B2000F0000E944209FF91EF91BF91AF919F9108
:101B30008F917F916F915F914F913F912F910F9076
:101B40000FBE0F901F9018951F920F920FB60F9215
:101B500011242F933F934F935F936F937F938F93B2
:101B60009F93AF93BF93CF93DF93EF93FF93C09176
:101B7000E900CF708091EC00D82FD17080FDD0E8C3
:101B80001092E9008091F000877F8093F0007894B4
:101B90000E94E80D1092E9008091F0008860809327
:101BA000F000CD2BCF70C093E900FF91EF91DF9152
:101BB000CF91BF91AF919F918F917F916F915F91E5
:101BC0004F913F912F910F900FBE0F901F9018953E
:101BD0001F93CF93DF93CDB7DEB7AA970FB6F894D4
:101BE000DEBF0FBECDBFEDE1F2E088E08E0F909139
:101BF000F10091938E13FBCF0E9461098091E80060
:101C000083FF1FC180911D0290911E02492F50E059
:101C10004A30510508F015C1FA01EA5AFF4F0C94F9
:101C20007024803881F0823809F00BC18091210244
:101C30008F708093E9008091EB0085FB882780F905
:101C40001092E90006C08091190290911A02911138
:101C500082609091E800977F9093E8008093F10074
:101C60001092F100C8C0282F2D7F09F0EAC0882308
:101C700019F0823061F0E5C080911F02813009F0D7
:101C8000E0C0933009F080E080931A022BC080916D
:101C90001F02811127C0809121028F7009F4D1C0E9
:101CA0008093E9002091EB0020FF1CC0933021F4C9
:101CB0008091EB00806214C09091EB009061909352
:101CC000EB0021E030E0A90102C0440F551F8A95C6
:101CD000E2F74093EA001092EA008091EB008860FE
:101CE0008093EB001092E9008091E800877F86C026
:101CF0008111A7C010911F021F778091E3008078A7
:101D0000812B8093E3008091E800877F8093E80037
:101D10000E94060C8091E80080FFFCCF8091E300D8
:101D200080688093E300111102C082E001C083E06B
:101D300080931C0286C08058823008F082C0809157
:101D40001F02909120028C3D53E0950779F583E0C6
:101D50008A838AE289834FB7F894DE01139620E0E4
:101D60003EE051E2E32FF0E050935700E49120FF72
:101D700003C0E295EF703F5FEF708E2F90E0EA3086
:101D800010F0C79601C0C0968D939D932F5F2431AC
:101D900049F74FBF8091E800877F8093E8006AE2AF
:101DA00070E0CE0101960E940D0B14C0AE014F5F92
:101DB0005F4F609121020E94540ABC01892B09F4F3
:101DC00040C09091E800977F9093E80089819A81C4
:101DD0000E94700B8091E8008B778093E80031C0FF
:101DE000803879F58091E800877F8093E8008091C2
:101DF00018028093F1008091E8008E778093E800CC
:101E00000E94060C1EC081111CC090911F029230CE
:101E1000C0F48091E800877F8093E80090931802D7
:101E20000E94060C80911802811106C08091E30087
:101E300087FD02C081E001C084E080931C020E9403
:101E40004D098091E80083FF0AC08091E800877FF8
:101E50008093E8008091EB0080628093EB00AA966B
:101E60000FB6F894DEBF0FBECDBFDF91CF911F91AB
:101E700008950895CF9380911C028823A1F0C0910A
:101E8000E900CF709091EC00892F817090FD80E87F
:101E9000C82B1092E9008091E80083FD0E94E80DB4
:101EA000CF70C093E900CF9108959093690180931A
:101EB00068010895E0916801F0916901309721F07F
:101EC0000190F081E02D099480E00895E09168018F
:101ED000F0916901309721F00280F381E02D09949F
:101EE0000895E0916801F0916901309721F0048034
:101EF000F581E02D099408952091660130916701E4
:101F00008217930771F09093670180936601E091C7
:101F10006801F0916901309721F00680F781E02D8A
:101F20000994089520916401309165018217930707
:101F300071F09093650180936401E0916801F091E4
:101F40006901309721F00084F185E02D099408950E
:101F500008950C94A80F0E943D1C0E9468040C94E4
:101F6000031DCF92DF92EF92FF920F931F93CF93B7
:101F7000DF93CDB7DEB72B970FB6F894DEBF0FBE59
:101F8000CDBF0E9480048BE6C82E81E0D82E00E0F1
:101F900010E0E02E802F0E946E05F60141916F0146
:101FA000F42EF826B1F40F5F1F4F0E30110589F79C
:101FB0008FEF89838A831B820E94461C8160782F61
:101FC0009D838C8349815A816B818D810E9454103D
:101FD00040C09091050291FF04C08B870E94740558
:101FE0008B8520E030E04F2D50E0922FBA01022E79
:101FF00002C0759567950A94E2F760FF24C02E83AE
:10200000EF8221E030E0690102C0CC0CDD1C9A9522
:10201000E2F790E08C219D21892B09F420E02887AC
:102020000E94461C8160782F9A8789874E815F8144
:1020300068858A850E945410F801E559FE4F808119
:10204000C826C08206C02F5F3F4F2630310569F693
:10205000AACF0E94EA1F10916A010E945A0F181716
:10206000A1F00E945A0F80936A012B960FB6F89444
:10207000DEBF0FBECDBFDF91CF911F910F91FF90BB
:10208000EF90DF90CF900C9450082B960FB6F894F9
:10209000DEBF0FBECDBFDF91CF911F910F91FF909B
:1020A000EF90DF90CF900895CF93DF93CDB7DEB759
:1020B0002B970FB6F894DEBF0FBECDBF4F83588766
:1020C00069877A878B87DE01119686E0FD01119280
:1020D0008A95E9F785E0FE01379601900D928A9581
:1020E000E1F749815A816B817C818D819E810E94BB
:1020F00084172B960FB6F894DEBF0FBECDBFDF91CD
:10210000CF9108950895CF93882309F4C2C0C82FB2
:10211000823859F40E945A0F81FDBBC089E30E94A6
:10212000A91A0E94761B89E30CC0833879F40E94B7
:102130005A0F80FDAEC083E50E94A91A0E94761B4B
:1021400083E50E94EB1ACF910C94761B843859F4E6
:102150000E945A0F82FD9DC087E40E94A91A0E9426
:10216000761B87E4EECF8CEF8C0F813A48F48C2FEE
:102170000E942C2281118DC08C2F0E94A91AE3CFBE
:1021800080E28C0F883048F4C77081E001C0880F6E
:10219000CA95EAF70E942F1BD6CF8BE58C0F8330B0
:1021A00078F4C53A29F0C63A31F083E890E005C0EA
:1021B00081E890E002C082E890E0CF910C947C0F1F
:1021C00088E58C0F833108F064C0C83A39F1C93A08
:1021D00041F1CA3A49F1CB3A51F1CC3A59F1CD3AF1
:1021E00061F1C03B69F1CE3A71F1CF3A79F1C13B6F
:1021F00081F1C23B89F1C33B91F1C43B99F1C53BED
:10220000A1F1C63BA9F1C73BB1F1C83BB9F1C93B4C
:10221000C1F1CA3BC9F180E090E038C082EE90E0A5
:1022200035C089EE90E032C08AEE90E02FC085EB99
:1022300090E02CC086EB90E029C087EB90E026C0B0
:102240008CEC90E023C08DEC90E020C083E891E01E
:102250001DC08AE891E01AC082E991E017C084E9C4
:1022600091E014C081E292E011C083E292E00EC0DE
:1022700084E292E00BC085E292E008C086E292E040
:1022800005C087E292E002C08AE292E0CF910C940E
:10229000920FCF910895882309F44BC0823859F4E6
:1022A0000E945A0F81FF45C089E30E94A91A0E942B
:1022B000761B89E30CC0833871F40E945A0F80FFAB
:1022C00038C083E50E94A91A0E94761B83E50E940C
:1022D000EB1A0C94761B843859F40E945A0F82FF33
:1022E00028C087E40E94A91A0E94761B87E4EFCFDA
:1022F0009CEF980F913A58F390E2980F983050F471
:10230000877091E001C0990F8A95EAF7892F0E94A2
:10231000351BDFCF9BE5980F933020F480E090E0F1
:102320000C947C0F885A833120F480E090E00C9468
:10233000920F0895882321F00E942F1B0C94761B86
:102340000895882321F00E94351B0C94761B089574
:10235000BF92CF92DF92EF92FF920F931F93CF9392
:10236000DF9300D000D000D0CDB7DEB725E0FC0170
:10237000DE01119601900D922A95E1F7FC01D080C3
:1023800011810281258122952F7043815481452B33
:1023900009F4FCC21F3F21F4FFEFDF1609F4F6C277
:1023A0007C012E830E948210D9821A8369817A81EE
:1023B000802F0E94861A182FB92E0E94DE190E94C3
:1023C000A5182E81002319F00E944C1B2E81EB2DA5
:1023D000E295EF70F0E0E05AFF4F0C9470248B2DE3
:1023E000807F9B2D9F70F92E882319F0F29480EF47
:1023F000F822002389F0FF2009F475C280E2810FE2
:10240000883020F48F2D0E942F1B03C08F2D0E9437
:102410003F1B0E94761B67C2812F0E944B11FF2039
:1024200009F4B4C2105E8F2D183018F40E94351BC9
:1024300002C00E94451B26960FB6F894DEBF0FBE61
:10244000CDBFDF91CF911F910F91FF90EF90DF9063
:10245000CF90BF900C94761B3B2D307F8B2D8F70CF
:10246000303211F08295807F112319F0113021F163
:102470002CC00023B9F0222309F4A0C1213009F0B7
:102480009DC126960FB6F894DEBF0FBECDBFDF917B
:10249000CF911F910F91FF90EF90DF90CF90BF9061
:1024A0000C945F1B222319F0213009F46FC28E8334
:1024B0000E94621B8E8196C1002321F0223008F019
:1024C00065C27CC1211162C28DC1002321F022238B
:1024D00009F474C108C2222309F484C119C22B2D46
:1024E00026952695237030E02115310521F0213005
:1024F0003105D1F04BC2002321F0812F9B2D937029
:1025000002C080E090E026960FB6F894DEBF0FBEC2
:10251000CDBFDF91CF911F910F91FF90EF90DF9092
:10252000CF90BF900C947C0F002321F0812F9B2D26
:10253000937002C080E090E026960FB6F894DEBF5C
:102540000FBECDBFDF91CF911F910F91FF90EF9004
:10255000DF90CF90BF900C94920F812F002319F041
:102560000E94F21E02C00E945A1F26960FB6F894CF
:10257000DEBF0FBECDBFDF91CF911F910F91FF90B6
:10258000EF90DF90CF90BF900C94DF1F8B2D837066
:1025900009F07BC00111FAC1812F82958695877061
:1025A000880F880F912F9F70C92ED12CE12CF12C10
:1025B000082E04C0CC0CDD1CEE1CFF1C0A94D2F7C4
:1025C00014FF12C04FE050E060E070E004C0440F20
:1025D000551F661F771F8A95D2F7CB01BA01609508
:1025E00070958095909503C060E070E0CB012B2D35
:1025F000269526952370422F50E042305105D9F0A0
:102600004330510569F16C297D298E299F2941307C
:10261000510551F126960FB6F894DEBF0FBECDBF1F
:10262000DF91CF911F910F91FF90EF90DF90CF90AE
:10263000BF900C94CC186C297D298E299F29269651
:102640000FB6F894DEBF0FBECDBFDF91CF911F91C3
:102650000F91FF90EF90DF90CF90BF900C94E8180F
:102660000E94CC18C701B60126960FB6F894DEBFBB
:102670000FBECDBFDF91CF911F910F91FF90EF90D3
:10268000DF90CF90BF900C94B018002319F08B2DE1
:10269000817001C08695882309F478C1812F8295C5
:1026A00086958770880F880F912F9F70C92ED12C27
:1026B000E12CF12C082E04C0CC0CDD1CEE1CFF1C00
:1026C0000A94D2F714FF12C04FE050E060E070E0CF
:1026D00004C0440F551F661F771F8A95D2F7CB01A0
:1026E000BA01609570958095909503C060E070E0A8
:1026F000CB012B2D269526952370422F50E042309A
:102700005105D9F04330510569F16C297D298E2995
:102710009F294130510551F126960FB6F894DEBF3E
:102720000FBECDBFDF91CF911F910F91FF90EF9022
:10273000DF90CF90BF900C94A6196C297D298E292B
:102740009F2926960FB6F894DEBF0FBECDBFDF914E
:10275000CF911F910F91FF90EF90DF90CF90BF909E
:102760000C94C2190E94A619C701B60126960FB68D
:10277000F894DEBF0FBECDBFDF91CF911F910F91B7
:10278000FF90EF90DF90CF90BF900C948A19103F8C
:10279000D1F118F4103E50F4A1C0123F09F463C007
:1027A00008F44CC0133F09F473C098C01F708B2D00
:1027B0008F710023A1F00E942319812F26960FB656
:1027C000F894DEBF0FBECDBFDF91CF911F910F9167
:1027D000FF90EF90DF90CF90BF900C949A110E94E1
:1027E0004419812F26960FB6F894DEBF0FBECDBFD9
:1027F000DF91CF911F910F91FF90EF90DF90CF90DD
:10280000BF900C94A1110023A9F02111BFC08B2D02
:102810008F7126960FB6F894DEBF0FBECDBFDF9145
:10282000CF911F910F91FF90EF90DF90CF90BF90CD
:102830000C946919223008F0A9C0E9CF0023A9F04F
:102840008B2D8F7126960FB6F894DEBF0FBECDBFCD
:10285000DF91CF911F910F91FF90EF90DF90CF907C
:10286000BF900C942319002359F38B2D8F7126965A
:102870000FB6F894DEBF0FBECDBFDF91CF911F9191
:102880000F91FF90EF90DF90CF90BF900C94441980
:10289000002399F08B2D8F7126960FB6F894DEBF2A
:1028A0000FBECDBFDF91CF911F910F91FF90EF90A1
:1028B000DF90CF90BF900C940E1926960FB6F89427
:1028C000DEBF0FBECDBFDF91CF911F910F91FF9063
:1028D000EF90DF90CF90BF900C9404190023A9F0E3
:1028E000222309F4ADCF812F26960FB6F894DEBFD0
:1028F0000FBECDBFDF91CF911F910F91FF90EF9051
:10290000DF90CF90BF900C948310222309F4ADCFB9
:10291000812F26960FB6F894DEBF0FBECDBFDF9194
:10292000CF911F910F91FF90EF90DF90CF90BF90CC
:102930000C944B114B2D4F70612FC7010E94040363
:1029400026960FB6F894DEBF0FBECDBFDF91CF91B4
:102950001F910F91FF90EF90DF90CF90BF900C945C
:1029600028184B2D4F70612FC70126960FB6F8948B
:10297000DEBF0FBECDBFDF91CF911F910F91FF90B2
:10298000EF90DF90CF90BF900C94750526960FB610
:10299000F894DEBF0FBECDBFDF91CF911F910F9195
:1029A000FF90EF90DF90CF90BF9008950E944C1B56
:1029B0000E945C1B0E94211B0E94761B0E948F209C
:1029C0000E94DF1F80E090E00E947C0F80E090E09A
:1029D0000C94920F0E943C1B0C94D6140E947B1AFC
:1029E000292F22952F7030E02C3031054CF42A30FD
:1029F00031056CF4225031092230310588F407C0CA
:102A00002C30310549F02F30310531F009C0803EBE
:102A100048F0803F29F406C093FB882780F9089589
:102A200080E0089581E00895CF93DF9300D000D037
:102A30001F92CDB7DEB70F900F900F900F900F90B1
:102A4000DF91CF910895CF93DF9300D000D000D0D5
:102A5000CDB7DEB726960FB6F894DEBF0FBECDBF5A
:102A6000DF91CF9108951F93CF93DF93C0917A01A7
:102A700016E080917B01C81799F0D0E01C9FF0010F
:102A80001D9FF00D1124E458FE4F40815181628159
:102A90007381848195810E9423152196C770E9CFA7
:102AA000DF91CF911F9108954091AC015091AD01FC
:102AB0006091AE017091AF018091B0019091B10130
:102AC0000C9423158091B10182958F7009F054C048
:102AD0008091AE01882309F44FC080917A01A091C2
:102AE0007B016091AC017091AD014091AF015091BB
:102AF000B001B6E08A1709F43FC090E041155105D6
:102B0000C1F17F3F11F46F3FA1F1B89FF001B99F70
:102B1000F00D1124E458FE4F218172132AC0208148
:102B2000621327C02281211124C0238134812417FC
:102B3000350710F421503109241B350B283C310591
:102B4000C0F42091B1012F7020612093B10126E0E3
:102B5000289FF001299FF00D1124EF57FE4F80812F
:102B60008F70806180838CEA91E00E94A8110C94A0
:102B7000331501968770BECF0895CF92DF92EF9202
:102B8000FF920F931F93CF93DF93CDB7DEB762977A
:102B90000FB6F894DEBF0FBECDBF8C0185E0F80103
:102BA000DE011D9601900D928A95E1F7D8014C91B6
:102BB00011965C91119712966C9112971396CD9085
:102BC000DC9014973091AC017091AD018091AF0110
:102BD0009091B001009709F46BC17F3F19F43F3F1A
:102BE00009F466C1E090AE01EE2009F4C0C0209166
:102BF000B101C816D90628F0F601E81BF90BCF0180
:102C000004C0809590958C0D9D1DFF24F394883C05
:102C1000910578F0F12C207F09F0C6C07C2DD98A6F
:102C2000C88A89890E9414158CEA91E00E94A81133
:102C3000B1C0822F807F09F046C0751314C03413D1
:102C400012C0611110C02F7020612093B1010E9449
:102C500054158CEA91E00E94A8118091B101D8012D
:102C600015968C932EC0CD2819F15F3F11F44F3F7C
:102C7000F9F0F62E61111CC080917A0120917B0140
:102C800036E0821709F45AC090E0389FF001399F6E
:102C9000F00D1124E458FE4F7181571306C0708166
:102CA000471303C07281711103C001968770E9CF89
:102CB000F62E662309F418C18091B10181608093DA
:102CC000B101F12C11C1751308C0341306C0611194
:102CD00004C08091B101D801C3C04D875E878D8546
:102CE0009E856A8B0E94EE146A898823E1F166232F
:102CF000D1F12091B101822F82958F7090E00297DF
:102D000074F08091AC019091AD0198878F83198602
:102D1000DB86CA862C87CE0107960E94A81186E022
:102D2000F801ACEAB1E001900D928A95E1F70E94BA
:102D300062150E945415FF24F394D6C04D875E8718
:102D40008D859E850E947B1A292F22952F7030E059
:102D5000223031050CF0BCC09F7009F0B6C0805E17
:102D6000883008F4C1C0C8010E94A811E4CFC81679
:102D7000D90608F453C0F601E81BF90BCF01883CD3
:102D8000910508F450C0F12C7C2DD98AC88A898914
:102D90000E941415ECEAF1E086E0DF011D928A95AD
:102DA000E9F70E945415A0C0751314C0341312C063
:102DB000611110C08091B101F8018583C8010E94A2
:102DC000A81186E0ECEAF1E0DF011D928A95E9F7AF
:102DD000FE2C8AC04D875E878D859E856A8B0E94FA
:102DE000EE146A89882309F4BECF662309F4BBCFA9
:102DF0002091B101822F82958F7090E002970CF4A0
:102E00008ECF8091AC019091AD019A8389831B8212
:102E1000DD82CC822E83CE0101967FCF8095909566
:102E20008C0D9D1DACCFF62E662309F49CCF751337
:102E30002EC034132CC02091B10120FD1FC0822F61
:102E400082958F70D9F0D80115962C9315978F30F5
:102E500049F08F5F982F9295907F822F8F70892BEA
:102E600015968C93C8010E94A81186E0F801ACEA7F
:102E7000B1E001900D928A95E1F793CF86E0F801D9
:102E8000ACEAB1E001900D928A95E1F72DC04D8733
:102E90005E878D859E850E94EE14811140CF8091C2
:102EA000B10181608093B101C8010E94A8111CC0CA
:102EB000662309F458CF4D875E878D859E850E94D5
:102EC000EE14882309F44FCF2ACF811148CF0CC0CC
:102ED000243031050CF047CF9F7009F440CFF80142
:102EE0009581907F09F03BCF8F2D62960FB6F894B5
:102EF000DEBF0FBECDBFDF91CF911F910F91FF902D
:102F0000EF90DF90CF9008951F93CF93DF93CDB7CD
:102F1000DEB72C970FB6F894DEBF0FBECDBF4F8340
:102F2000588769877A878B879C87CE0107960E948E
:102F3000BD15882369F08F8198852A853B85232BD1
:102F4000F1F19F3F09F063C08F3F09F060C037C0C7
:102F500086E0FE013796DE01119601900D928A956A
:102F6000E1F76F817885EA85FB85309741F17F3FF6
:102F700011F46F3F21F120917B0130E0C9010196EE
:102F80008770992740917A0150E08417950709F4DA
:102F900047C069837A83FD83EC8396E0929FD001DA
:102FA000939FB00D1124A458BE4FFE01319601909D
:102FB0000D929A95E1F780937B010E94331516E0FC
:102FC00080917A0190917B018917C1F1189FC0010E
:102FD000112484589E4F0E94BD15882379F1E091F9
:102FE0007A011E9FF0011124E458FE4F4081518167
:102FF00062817381848195810E94231580917A0179
:1030000090E001968770992780937A01D9CF4F81FC
:10301000588569857A858B859C850E942315CFCF3D
:103020000E94EA1410927B0110927A01ECEAF1E01E
:1030300086E0DF011D928A95E9F7C1CF2C960FB685
:10304000F894DEBF0FBECDBFDF91CF911F910895E1
:10305000EF92FF920F931F93CF93DF938C01892BF5
:1030600009F46CC0F12CEE24E394E8012196F801F8
:103070008491843740F4843008F051C0813081F06D
:10308000823019F15BC0853709F444C0A8F19CE790
:10309000980F903708F052C08F770E944B1141C0B3
:1030A0000E5F1F4FFE01C49180E28C0F883048F400
:1030B000C7708E2D01C0880FCA95EAF70E944F1B7A
:1030C00014C08C2F0E9483102DC00E5F1F4FFE0175
:1030D000C49180E28C0F883058F4C7708E2D01C0E7
:1030E000880FCA95EAF70E94551B0E94761B1AC0EA
:1030F0008C2F0E944B1116C00E5F1F4FFE01C49112
:10310000CC2381F08FE99FE00197F1F700C0000028
:10311000C150F6CF0E5F1F4FFE01F49003C00E9416
:1031200083108E018F2D882309F49FCFEFE9FFE0F4
:103130003197F1F700C000008150F5CFDF91CF91BA
:103140001F910F91FF90EF90089508956093ED0106
:103150007093EE018093EF019093F0010C94D614DC
:103160000F931F930091ED011091EE012091EF015B
:103170003091F001DC01CB01802B912BA22BB32BE2
:103180008093ED019093EE01A093EF01B093F001D5
:103190001F910F910C94D6140F931F930091ED0182
:1031A0001091EE012091EF013091F001DC01CB0193
:1031B00080239123A223B3238093ED019093EE010A
:1031C000A093EF01B093F0011F910F910C94D614CE
:1031D0000F931F930091ED011091EE012091EF01EB
:1031E0003091F001DC01CB0180279127A227B32782
:1031F0008093ED019093EE01A093EF01B093F00165
:103200001F910F910C94D6141092E9011092EA01CB
:103210001092EB011092EC010C94D61441E050E0B6
:1032200060E070E004C0440F551F661F771F8A9549
:10323000D2F74093E9015093EA016093EB01709358
:10324000EC010C94D61441E050E060E070E004C062
:10325000440F551F661F771F8A95D2F78091E901A9
:103260009091EA01A091EB01B091EC01482B592B10
:103270006A2B7B2B4093E9015093EA016093EB01A9
:103280007093EC010C94D61441E050E060E070E0E3
:1032900004C0440F551F661F771F8A95D2F74095CB
:1032A0005095609570958091E9019091EA01A09107
:1032B000EB01B091EC01482359236A237B2340930F
:1032C000E9015093EA016093EB017093EC010C94D7
:1032D000D61441E050E060E070E004C0440F551F98
:1032E000661F771F8A95D2F78091E9019091EA01D4
:1032F000A091EB01B091EC01482759276A277B2761
:103300004093E9015093EA016093EB017093EC0163
:103310000C94D6140F931F930091E9011091EA01C8
:103320002091EB013091EC01DC01CB01802B912B42
:10333000A22BB32B8093E9019093EA01A093EB01B8
:10334000B093EC011F910F910C94D6140F931F931F
:103350000091E9011091EA012091EB013091EC011B
:10336000DC01CB0180239123A223B3238093E901C5
:103370009093EA01A093EB01B093EC011F910F91A0
:103380000C94D6140F931F930091E9011091EA0158
:103390002091EB013091EC01DC01CB0180279127DA
:1033A000A227B3278093E9019093EA01A093EB0150
:1033B000B093EC011F910F910C94D6140895292F0E
:1033C000220F920F990F890FA82FA695A695A69563
:1033D000877051E001C0550F8A95EAF785E0A89FF4
:1033E000D001112420E030E070E0F901EA0FFB1F6A
:1033F000EE54FE4F4081CB01022E02C09695879578
:103400000A94E2F781709927819584278523842780
:1034100080832F5F3F4F2530310539F70895292FDD
:10342000220F920F990F890F682F66956695669502
:10343000982F977085E0689FB001112440E050E01C
:1034400080E0FA01E60FF71FEE54FE4F208130E0D6
:10345000092E02C0369527950A94E2F7217033278A
:10346000042E01C0220F0A94EAF7822B4F5F5F4FB0
:103470004530510531F70895CF92DF92EF92FF92D8
:103480000F931F93CF93DF938C01C090ED01D090E9
:10349000EE01E090EF01F090F0018091E901909150
:1034A000EA01A091EB01B091EC01C82AD92AEA2ADD
:1034B000FB2ACFE1D0E0D701C6010C2E04C0B6959F
:1034C000A795979587950A94D2F780FF06C0B80113
:1034D0008C2F0E94B507019721F4219760F780E0B7
:1034E00001C08C2FDF91CF911F910F91FF90EF9032
:1034F000DF90CF900895CF93DF93EC010E943C1AA8
:10350000BE010E94B507DF91CF9108951F93CF931D
:10351000DF93EB0190917901992321F0CB010E9477
:103520007B1A13C0882349F0CB010E943C1A182F44
:10353000682FCE010E94DF1904C0CB010E940F1A30
:10354000182FBE01812F0E94B507DF91CF911F91E7
:10355000089590910C01992321F090910D01911102
:1035600009C020910E0130910F01F90132969FEFB1
:1035700040E01FC0982F9695969596959F3050F5F0
:10358000E0910E01F0910F01E90FF11D877021E02C
:1035900030E0A90102C0440F551F8A95E2F7CA0125
:1035A0009181892B818308959F3F39F04F5F4E3081
:1035B00041F051915813F8CF0DC05111F7CF942F0E
:1035C000F5CF9F3F39F0F901E90FF11D97FDFA950D
:1035D00082830895089590910C01992321F0909190
:1035E0000D01911109C020910E0130910F01F901D7
:1035F0003296205F3F4F1FC0982F969596959695CF
:103600009F30F0F4E0910E01F0910F01E90FF11DF0
:10361000877021E030E0A90102C0440F551F8A9550
:10362000E2F7CA01809591818923818308953196BB
:10363000E217F30729F090819813F9CF1082F7CFA2
:10364000089581E090E0E0910E01F0910F01E80F04
:10365000F91F1082019680319105A9F70895909184
:103660000402892B809304020895809590910402AE
:103670008923809304020895109204020895909182
:103680000302892B80930302089580959091030291
:103690008923809303020895109203020895909164
:1036A0000202892B80930202089580959091020274
:1036B0008923809302020895109202020895809354
:1036C000F10108951092F101089580910E019091F9
:1036D0000F01FC0131969C01205F3F4F80E09191EA
:1036E00091118F5FE217F307D1F70895E0910E0172
:1036F000F0910F01809104028083E0910E01F0911E
:103700000F01908180910302892B8083E0910E014B
:10371000F0910F01908180910202892B808380912A
:10372000F101882361F0E0910E01F0910F01908189
:10373000892B80830E94651B81111092F101809179
:103740000E0190910F010C94660FCF92DF92EF92D1
:10375000FF926C01EE24FF24C114D104E104F104B2
:1037600021F0C701B60120E101C020E0C72ED82E0C
:10377000E92EFF24C114D104E104F10419F0285FFB
:10378000C701B6016B017C0154E0F694E794D7942D
:10379000C7945A95D1F7C114D104E104F10419F08A
:1037A0002C5FC701B6016B017C0142E0F694E794FF
:1037B000D794C7944A95D1F7C114D104E104F10418
:1037C00019F02E5FC701B601DC01CB01B695A795B4
:1037D00097958795892B8A2B8B2B09F02F5F822F4A
:1037E000FF90EF90DF90CF90089580911C0284307D
:1037F00039F11092060220E488E190E00FB6F894C7
:10380000A895809360000FBE2093600080E00E9426
:10381000500883B7817F846083BF83B7816083BF93
:103820007894889583B78E7F83BF0FB6F894A89558
:1038300080916000886180936000109260000FBEEC
:10384000089508950895CF930E94211C0E9480043A
:103850000E94221CC0E08C2F0E946E05811104C0C2
:10386000CF5FCE30C1F701C081E0CF9108950E94B3
:10387000EA140E945A0F0C94500882E084BD93E031
:1038800095BD9AEF97BD80936E0008952FB7F89479
:103890008091070290910802A0910902B0910A025A
:1038A0002FBF0895CF92DF92EF92FF920F931F9355
:1038B0002FB7F894409107025091080260910902D5
:1038C00070910A022FBF6A017B01EE24FF248C0154
:1038D00020E030E0C016D106E206F30610F44150B5
:1038E00051099A01281B390BC9011F910F91FF90B3
:1038F000EF90DF90CF9008951F920F920FB60F9226
:1039000011248F939F93AF93BF938091070290915F
:103910000802A0910902B0910A020196A11DB11DF1
:103920008093070290930802A0930902B0930A02C1
:10393000BF91AF919F918F910F900FBE0F901F90ED
:1039400018950E94570CF8942FEF87EA91E62150C2
:1039500080409040E1F700C0000087E090EBDC0180
:103960008093260290932702A0932802B093290205
:103970009CE088E10FB6F894A895809360000FBE94
:1039800090936000FFCFEF92FF920F931F93CF931E
:10399000DF93D82FC0E08C2F0E946E0500E010E06E
:1039A000E82EF12CC701002E02C0959587950A9448
:1039B000E2F780FD06C00F5F1F4F0630110591F73B
:1039C00009C0602F7C2F80E00E947605D813F3CFCA
:1039D00081E004C0CF5FCE30F1F680E0DF91CF917F
:1039E0001F910F91FF90EF900895CF93C82F8CE215
:1039F0000E94C31C882321F08C2FCF910C94C31CF0
:103A000080E0CF910895CF930E944A1E811102C099
:103A10000E94301EC5E6C15049F00E9480048FE329
:103A20009CE90197F1F700C00000F5CF89E20E9400
:103A3000F51C811113C18AE20E94F51C81110E94BC
:103A4000301E85E00E94F51C81110E94A11C0E947D
:103A5000551E8093050287E00E94F51C8823A9F17A
:103A60008BE10E94F51C882351F08091050281FBB7
:103A7000222720F991E0922790FB81F90EC08EE079
:103A80000E94F51C882361F08091050282FB2227A9
:103A900020F991E0922790FB82F98093050215C0EE
:103AA00080E10E94F51C90910502882341F093FB70
:103AB000222720F981E0822780FB93F904C0892F17
:103AC000809580FB90F990930502809105020E94F9
:103AD000591E0E94671E8093250280EE0E94F51CED
:103AE000882341F080912502982F909590FB80F9D2
:103AF0008093250289E30E94F51C882359F0809168
:103B0000250281FB222720F991E0922790FB81F981
:103B10008093250282EE0E94F51C882359F0809143
:103B2000250282FB222720F991E0922790FB82F95F
:103B30008093250286EE0E94F51C882359F080911F
:103B4000250283FB222720F991E0922790FB83F93D
:103B50008093250283EE0E94F51C882359F0809102
:103B6000250284FB222720F991E0922790FB84F91B
:103B70008093250285E30E94F51C882359F08091EB
:103B8000250285FB222720F991E0922790FB85F9F9
:103B90008093250281E30E94F51C882359F08091CF
:103BA000250286FB222720F991E0922790FB86F9D7
:103BB0008093250281E10E94F51C882359F08091B1
:103BC000250287FB222720F991E0922790FB87F9B5
:103BD00080932502809125020E946B1E8091250210
:103BE00087FB882780F980930D0187E20E94F51CEE
:103BF000C82F8EE10E94F51C8111C2608FE10E94E6
:103C0000F51C8111C46080E20E94F51C8111C8601E
:103C100081E20E94F51C8111C06182E20E94F51CC4
:103C20008111C06283E20E94F51C8111C06484E2AC
:103C30000E94F51C882311F0C06802C0CC2329F033
:103C40008C2F0E94621E6C2F03C00E945E1E682F84
:103C500070E080E090E0CF910C94A618CF91089589
:103C60006DEE7EEF80E090E00E94AA2460E082E0AA
:103C700090E00E94982460E083E090E00E94982405
:103C800060E084E090E00E94982460E085E090E0AD
:103C90000C94982480E090E00E94922421E08D3ED4
:103CA0009E4F09F020E0822F089582E090E00C946E
:103CB0008A24682F82E090E00C94982483E090E0BE
:103CC0000C948A24682F83E090E00C94982484E07C
:103CD00090E00C948A24682F84E090E00C9498245F
:103CE00080910D0280FF0BC06091130185E0689FF9
:103CF000B001112475956795759567952BC081FF67
:103D000009C06091130185E0689FB0011124759589
:103D1000679520C082FF07C06091130185E0689F0E
:103D2000B001112417C090910E029923D1F0609137
:103D30001201961788F72091130185E0289F9001C2
:103D40001124929FA001939F500D112470E0CA018D
:103D50000E945C246038710540F46115710539F0EA
:103D600002C065E070E0862F08958FE7089581E036
:103D7000089580910D0280FF08C06091110170E0EC
:103D8000759567957595679521C081FF06C060910F
:103D9000110170E07595679519C082FF04C06091AC
:103DA000110170E010C090910E029923C1F0609152
:103DB00010019617A0F780911101899FC00111246D
:103DC00070E00E945C246038710528F4611571056B
:103DD00021F0862F08958FE7089581E0089561E02E
:103DE00070E0F4CF803F21F40E94701E819504C0E2
:103DF000813F29F40E94701E809311020895823F32
:103E000021F40E94701E819504C0833F29F40E9412
:103E1000701E809310020895893F19F40E94B91E04
:103E200005C08A3F31F40E94B91E81958093120229
:103E300008958B3F21F40E94B91E819504C08C3FE8
:103E400029F40E94B91E809313020895843F21F43F
:103E500080910F02816017C0853F21F480910F028D
:103E6000826011C0863F21F480910F0284600BC0F4
:103E7000873F21F480910F02886005C0883F31F4AC
:103E800080910F02806180930F0208958D3F21F48D
:103E900080910D0281600BC08E3F21F480910D0254
:103EA000826005C08F3F29F480910D028460809369
:103EB0000D020895803F39F48091110287FF6CC094
:103EC0001092110269C0813F29F4809111021816E5
:103ED000BCF362C090911002823F29F497FF5CC04E
:103EE0001092100259C0833F19F41916CCF354C034
:103EF000893F41F48091120218160CF04DC01092C7
:103F000012024AC08A3F29F48091120287FF44C0FE
:103F1000F6CF8B3F39F48091130287FF3DC010929A
:103F200013023AC08C3F29F4809113021816BCF397
:103F300033C0843F21F480910F028E7F17C0853FEC
:103F400021F480910F028D7F11C0863F21F4809172
:103F50000F028B7F0BC0873F21F480910F02877F78
:103F600005C0883F31F480910F028F7E80930F024D
:103F700013C08D3F21F480910D028E7F0BC08E3FC8
:103F800021F480910D028D7F05C08F3F29F480912F
:103F90000D028B7F80930D028091100281110EC063
:103FA0008091110281110AC080911202811106C014
:103FB00080911302811102C010920E0208958FE0C9
:103FC00092E00E94710F0E94461C90930C02809315
:103FD0000B0208951F93CF93DF9380910B02909172
:103FE0000C020E94521CAC0190910E02992321F008
:103FF0002091140130E006C0209115018AE0289F2D
:10400000900111244217530708F485C080911002D3
:10401000C0911102D091120210911302811107C0B8
:10402000C11175C0D11173C0111171C074C09F3F0F
:1040300019F09F5F90930E02181624F40E94701ED0
:10404000809310028091100287FF05C00E94701EAD
:104050008195809310021C1624F40E94701E809398
:1040600011028091110287FF05C00E94701E819588
:104070008093110260911002662331F1C091110208
:10408000CC2311F1062E000C770B880B990B0E94A4
:10409000632323E333E343E35FE30E94C7230E94E8
:1040A0002B23609310026C2FCC0F770B880B990B8E
:1040B0000E94632323E333E343E35FE30E94C723C8
:1040C0000E942B23609311021D1624F40E94B91E36
:1040D000809312028091120287FF05C00E94B91ED0
:1040E000819580931202111624F40E94B91E8093C8
:1040F00013028091130287FF05C00E94B91E8195AB
:1041000080931302DF91CF911F910C94DF1F9F3F8B
:1041100009F08FCF97CFDF91CF911F910895EFE0F6
:10412000F2E085E0DF011D928A95E9F710920E0218
:1041300010920D020895833081F128F4813059F0F6
:104140008230D1F00895853009F449C0B8F1863045
:1041500009F456C0089580911501262F30E0280FEC
:10416000311D2F3F310524F4680F60931501089528
:104170008FEF80931501089580911401262F30E070
:10418000280F311D2F3F310524F4680F609314016F
:1041900008958FEF80931401089580911301262FC5
:1041A00030E0280F311D2F3F310524F4680F609354
:1041B000130108958FEF80931301089580911201E8
:1041C000262F30E0280F311D2F3F310524F4680FD2
:1041D0006093120108958FEF8093120108958091EA
:1041E0001101262F30E0280F311D2F3F310524F417
:1041F000680F6093110108958FEF80931101089566
:1042000080911001262F30E0280F311D2F3F3105FE
:1042100024F4680F6093100108958FEF80931001CC
:104220000895833011F128F4813049F0823091F003
:104230000895853081F120F18630C1F10895809193
:104240001501681720F4861B8093150108951092BC
:104250001501089580911401681720F4861B80933E
:1042600014010895109214010895809113016817A4
:1042700020F4861B80931301089510921301089572
:1042800080911201681720F4861B80931201089513
:1042900010921201089580911101681720F4861B75
:1042A00080931101089510921101089580911001D9
:1042B000681720F4861B8093100108951092100156
:1042C00008950F931F938D3109F46BC008F03FC020
:1042D0008E3009F47FC0C0F4873009F469C068F4F7
:1042E000863009F0B1C080910502817F8E7F809376
:1042F000050281E080931502A8C0883009F4A2C0AD
:104300008B3009F49FC0A0C0863109F49BC078F4BB
:10431000803109F472C0813109F096C00E94EA141C
:1043200090910D0181E0892780930D018BC0893127
:1043300009F488C08B3109F087C08091050281FBA8
:10434000222720F991E0922790FB81F94CC0853318
:1043500009F470C048F4873209F46CC008F459C0FD
:10436000893209F467C070C0833438F48A3308F0A6
:104370004EC0883309F466C067C0833409F45AC05C
:10438000883409F061C00E94EA140FEF13ED20E3B6
:10439000015010402040E1F700C000000E94A11C25
:1043A00051C00E94E5220E945A0F0E9450084AC044
:1043B00090910502892F8095817080FB90F929F0FA
:1043C000966098609093050240C0997F977F909384
:1043D000050238C08091050282FB222720F991E076
:1043E000922790FB82F980930502992359F18091DD
:1043F000050281608093050225C08091050283FB40
:10440000222720F991E0922790FB83F9ECCF895382
:1044100001C08D5141E050E060E070E08A019B01F5
:1044200004C0000F111F221F331F8A95D2F7C90144
:10443000B80104C061E070E080E090E00E94A6183E
:104440000E94EA1481E001C080E01F910F9108955D
:1044500080E0089580E00895CF93C82F80911502E1
:10446000813079F018F08230E9F187C0E0910E01D7
:10447000F0910F018081813169F0823209F07FC0B3
:1044800009C0E0910E01F0910F018081813111F09E
:10449000823261F48C2F0E942822811104C08C2F5B
:1044A0000E9461211DC081E090E01AC08C2F0E9403
:1044B0002A22811114C0C43179F048F4CB3079F04C
:1044C000C03109F060C082E08093150208C0C93293
:1044D00019F0C83321F057C01092150254C081E082
:1044E000817053C0C93289F118F5C43171F1A8F453
:1044F000C73009F046C08AE08093150194E190939B
:10450000140193E0909313018093120188E080934B
:10451000110188E28093100134C0CE51C63088F575
:10452000EC2FF0E0E65DFE4F80818093140229C0FD
:10453000CE34E9F020F4CB3421F56AE013C0C13564
:1045400079F0C235F1F461E00DC080911402882346
:1045500019F01092140215C081E08093150215C065
:1045600061E006C0809114020E949B200AC06AE0AC
:10457000809114020E94112104C01092150280E063
:1045800004C081E002C080E0ABCFCF910895E1E8A4
:10459000F0E08081886080838081816080838FB734
:1045A000F89493E09093890090ED909388008FBFEA
:1045B0000895EFE6F0E08081826080830895EFE661
:1045C000F0E080818D7F80830895EFE6F0E09081B8
:1045D00082E08927808308951F920F920FB60F9271
:1045E00011242F933F934F935F936F937F938F93F8
:1045F0009F93AF93BF93EF93FF9380911602909197
:10460000170201969093170280931602811103C03E
:1046100082E00E945008E0911702E695E695F0E0EE
:10462000EA5CFA4FE491809116028E1303C080E099
:104630000E945008FF91EF91BF91AF919F918F9190
:104640007F916F915F914F913F912F910F900FBE8E
:104650000F901F9018950E9432236894B1110C940A
:10466000C12308950E94A62388F09F5798F0B92F80
:104670009927B751B0F0E1F0660F771F881F991F97
:104680001AF0BA95C9F714C0B13091F00E94C02356
:10469000B1E008950C94C023672F782F8827B85F66
:1046A00039F0B93FCCF3869577956795B395D9F7EF
:1046B0003EF490958095709561957F4F8F4F9F4FF9
:1046C0000895E89409C097FB3EF490958095709505
:1046D00061957F4F8F4F9F4F9923A9F0F92F96E94E
:1046E000BB279395F695879577956795B795F111C3
:1046F000F8CFFAF4BB0F11F460FF1BC06F5F7F4F60
:104700008F4F9F4F16C0882311F096E911C0772371
:1047100021F09EE8872F762F05C0662371F096E87A
:10472000862F70E060E02AF09A95660F771F881F49
:10473000DAF7880F9695879597F9089557FD905861
:10474000440F551F59F05F3F71F04795880F97FB55
:10475000991F61F09F3F79F087950895121613060F
:104760001406551FF2CF4695F1DF08C0161617063E
:104770001806991FF1CF8695710561050894089573
:10478000E894BB2766277727CB0197F908950E9405
:10479000DA230C944B240E943D2438F00E944424D8
:1047A00020F0952311F00C9434240C943A24112415
:1047B0000C94C1230E949E2370F3959FC1F3950F23
:1047C00050E0551F629FF001729FBB27F00DB11D95
:1047D000639FAA27F00DB11DAA1F649F6627B00D25
:1047E000A11D661F829F2227B00DA11D621F739F0E
:1047F000B00DA11D621F839FA00D611D221F749F1C
:104800003327A00D611D231F849F600D211D822F62
:10481000762F6A2F11249F5750409AF0F1F0882389
:104820004AF0EE0FFF1FBB1F661F771F881F9150B6
:104830005040A9F79E3F510580F00C9434240C940D
:10484000C1235F3FE4F3983ED4F38695779567954F
:10485000B795F795E7959F5FC1F7FE2B880F911DE0
:104860009695879597F9089597F99F6780E870E086
:1048700060E008959FEF80EC089500240A941616D6
:10488000170618060906089500240A94121613063E
:10489000140605060895092E0394000C11F48823CC
:1048A00052F0BB0F40F4BF2B11F460FF04C06F5FE8
:1048B0007F4F8F4F9F4F089597FB072E16F400945C
:1048C00007D077FD09D00E94762407FC05D03EF47E
:1048D000909581959F4F0895709561957F4F0895AC
:1048E000EE0FFF1F0590F491E02D0994AA1BBB1B4E
:1048F00051E107C0AA1FBB1FA617B70710F0A61BE0
:10490000B70B881F991F5A95A9F780959095BC0100
:10491000CD010895F999FECF92BD81BDF89A9927EE
:1049200080B50895A8E1B0E042E050E00C94B224D4
:10493000262FF999FECF92BD81BDF89A019700B458
:10494000021639F01FBA20BD0FB6F894FA9AF99AF8
:104950000FBE08950196272F0E9499240C94982445
:10496000DC01CB01FC01F999FECF06C0F2BDE1BD2F
:10497000F89A319600B40D9241505040B8F708951E
:04498000F894FFCFD9
:1049840020025208E008BD08890855080101F20117
:1049940028080A03140A3F4D3639F704AA0474049C
:1049A4003B04CE03E70300041904010203040506D3
:0449B40007080900E7
:00000001FF
